:100000000C94D6040C941D050C941D050C941D0530
:100010000C941D050C941D050C941D050C941D05D8
:100020000C941D050C941D050C94C21E0C94FE1D11
:100030000C9447260C941D050C941D050C941D056D
:100040000C941D050C941D050C941D050C941D05A8
:100050000C941D050C946E250C941D050C941D0527
:100060000C941D050C941D050C941D050C941D0588
:100070000C941D050C941D050C941D050C941D0578
:100080000C941D050C941D050C941D050C941D0568
:100090000C941D050C941D050C941D050C941D0558
:1000A0000C941D050C941D050C941D0520117F1149
:1000B000841189118E11931198119D11A211A7110C
:1000C000AC11B311B611B911BC11BF11C211C511D8
:1000D000C811CD118A128A12C412C4121713331315
:1000E000C514C5143E131C142D142D140C1C331CE4
:1000F000E01D331CE01D7F1CA21CE01DA31DB21DD2
:1001000035273527482748273E27482748274827A7
:100110003527352743274827482743270001010172
:1001200001010101010102020202020202020203B4
:100130000303030303030304040404040404050584
:100140000505050606060606070707070708080847
:1001500008090909090A0A0A0B0B0B0C0C0C0D0DF6
:100160000D0E0E0E0F0F0F1010111111121213138E
:100170001414151516161717181819191A1A1B1B07
:100180001C1D1D1E1E1F2020212222232424252663
:1001900026272829292A2B2C2D2D2E2F303132329B
:1001A000333435363738393A3B3C3D3E3F404142A7
:1001B000434445464748494A4C4D4E4F505153548D
:1001C000555658595A5B5D5E5F6162646566686941
:1001D0006B6C6D6F7072737577787A7B7D7E8082C1
:1001E000838587888A8C8E8F91939596989A9C9E0A
:1001F000A0A2A3A5A7A9ABADAFB1B3B5B7BABCBE1A
:10020000C0C2C4C6C9CBCDCFD1D4D6D8DBDDDFE2E6
:10021000E4E7E9EBEEF0F3F5F8FAFDFF7267626CE4
:10022000696768742074696D657220656E61626CBF
:1002300065642E0A007267626C69676874206D6F6E
:100240006465205B4E4F454550524F4D5D3A202529
:10025000750A007267626C69676874206D6F646507
:10026000205B454550524F4D5D3A2025750A00727E
:1002700067626C69676874207365742068737620A0
:100280005B4E4F454550524F4D5D3A2025752C250C
:10029000752C25750A007267626C69676874207333
:1002A000657420687376205B454550524F4D5D3A2A
:1002B0002025752C25752C25750A007267626C69DE
:1002C000676874207261696E626F7720736574204D
:1002D0006873763A2025642C25642C25642C2575BA
:1002E0000A00FFAA7F55407267626C6967687420D4
:1002F00074696D65722064697361626C652E0A00B1
:100300002223252628292A2C2D2F30323335363822
:100310003A3B3D3E4042434547494A4C4E5051537B
:100320005557595A5C5E6062646668696B6D6F719F
:10033000737577797B7D7F81838587898A8C8E90A1
:10034000929496989A9C9E9FA1A3A5A7A8AAACAEAA
:10035000AFB1B3B4B6B8B9BBBCBEBFC1C2C3C5C6EA
:10036000C7C9CACBCCCDCED0D1D2D2D3D4D5D6D793
:10037000D7D8D9D9DADADBDBDBDCDCDCDCDCDDDDD1
:10038000DDDDDCDCDCDCDCDBDBDBDADAD9D9D8D7C1
:10039000D7D6D5D4D3D2D2D1D0CECDCCCBCAC9C763
:1003A000C6C5C3C2C1BFBEBCBBB9B8B6B4B3B1AF9A
:1003B000AEACAAA8A7A5A3A19F9E9C9A989694923A
:1003C000908E8C8A89878583817F7D7B7977757311
:1003D000716F6D6B6968666462605E5C5A595755EF
:1003E0005351504E4C4A4947454342403E3D3B3AAB
:1003F0003836353332302F2D2C2A29282625232232
:100400007267626C696768742064697361626C65A5
:10041000205B454550524F4D5D3A207267626C69D2
:100420006768745F636F6E6669672E656E61626C84
:1004300065203D2025750A007267626C69676874E3
:1004400020656E61626C65205B454550524F4D5D85
:100450003A207267626C696768745F636F6E666981
:10046000672E656E61626C65203D2025750A0072FD
:1004700067626C6967687420746F67676C65205B7E
:10048000454550524F4D5D3A207267626C6967680E
:10049000745F636F6E6669672E656E61626C65205E
:1004A0003D2025750A0044454255473A206469734A
:1004B00061626C65642E0A0044454255473A2065E6
:1004C0006E61626C65642E0A0029001E001F002008
:1004D0000021002200230024002500260027002DF3
:1004E000002E00310035002B0014001A0008001502
:1004F0000017001C0018000C00120013002F003021
:10050000002A004C00015104001600070009000AEF
:10051000000B000D000E000F0033003400280028EF
:10052000004B00E1001D001B000600190005001132
:10053000001000360037003800E500E50052004E9C
:1005400000E000E200E3002C002C002C002C002C2A
:10055000002C00E600E400E400500051004F0000D1
:100560005C000000000000CC5CCB5C0000000000E0
:100570000000000000000000000000015C0000001E
:100580000000000000CA5CC95C0000000000000020
:10059000000000000000000000000001000000005A
:1005A000000000C85CC75C0000CD5CCE5CCF5CD0B6
:1005B0005CD15CD25CD35CD45C0000000000000025
:1005C00000C65CC55C0000000000000000000000E8
:1005D0000000000000000000000000C05CC25CC41D
:1005E0005CC35C0000000000000000000000000090
:1005F000000000DE5C7267626C696768745F636F3D
:100600006E6669672E7370656564203D2025640AF7
:10061000007267626C696768745F636F6E666967B2
:100620002E76616C203D2025640A007267626C6939
:100630006768745F636F6E6669672E736174203DCF
:100640002025640A007267626C696768745F636F73
:100650006E6669672E687565203D2025640A007204
:1006600067686C696768745F636F6E6669672E6D33
:100670006F6465203D2025640A007267626C6967BB
:1006800068745F636F6E6669672E656E61626C6524
:10069000203D2025640A007267626C696768745F98
:1006A000636F6E66696720454550524F4D3A0A00A8
:1006B0007267626C696768745F696E6974207267DB
:1006C000626C696768745F636F6E6669672E6D6FD1
:1006D0006465203D20302E20577269746520646562
:1006E0006661756C742076616C75657320746F201B
:1006F000454550524F4D2E0A007267626C6967681B
:10070000745F696E6974206565636F6E66696720E2
:100710006973206E6F7420656E61626C65642E0A69
:10072000007267626C696768745F696E69742073D0
:1007300074617274210A007267626C696768745F21
:10074000696E69742063616C6C65642E0A000A002E
:100750002530313662003A200025303258000A72C6
:100760002F63203031323334353637383941424304
:100770004445460A0032190A00047F3F1F643214C0
:10078000643214783C1E1E140A050A0025303258C3
:10079000006B6579626F6172645F7365745F6C652D
:1007A000643A20005B735D004B6579626F6172642F
:1007B0002073746172742E0A000631FF0974A1015E
:1007C0000975150026FF0095207508810209761528
:1007D0000026FF00952075089102C005010902A1BD
:1007E0000185020901A10005091901290515002546
:1007F00001950575018102950175038101050109C6
:100800003009311581257F95027508810609381553
:1008100081257F950175088106050C0A380215812E
:10082000257F950175088106C0C005010980A101D9
:10083000850319012AB700150126B7009501751027
:100840008100C0050C0901A101850419012AA0023B
:10085000150126A002950175108100C00501090649
:10086000A101050719E029E7150025019508750183
:1008700081029501750881010507190029FF1500FE
:1008800026FF0095067508810005081901290595C0
:100890000575019102950175039101C05B435D00EF
:1008A0005B445D005B535D005B575D005B525D0028
:1008B00009025B00030100A0FA0904000001030122
:1008C00001000921110100012240000705810308F0
:1008D000000A0904010001030000000921110100C0
:1008E000012281000705820320000A090402000298
:1008F00003000000092111010001222200070583E5
:10090000032000010705030320000112011001006C
:10091000000008646975000100010203010403304E
:100920000000000C03490064006F0062006F0000CB
:10093000001003470065006E0065007200690063E7
:10094000000000040309040A002530325820006B1F
:100950006579626F6172645F7265706F72743A205C
:1009600000290A002575002F002575005D28002547
:100970006400200025640020002564002000256418
:10098000007C0025303258006D6F7573656B65799A
:10099000205B62746E7C782079207620685D2872F6
:1009A00065702F61636C293A205B000011241FBE23
:1009B000CFEFDAE0DEBFCDBF04B603FE27C08091E3
:1009C0000A0390910B03A0910C03B0910D038730A3
:1009D000904BA740B04BD1F410920A0310920B0336
:1009E00010920C0310920D0314BE84B7877F84BF4E
:1009F0000FB6F894A895809160008861809360009C
:100A0000109260000FBEE0E0F8E3099511E0A0E06D
:100A1000B1E0E4ECF3E502C005900D92AC39B1070A
:100A2000D9F723E0ACE9B1E001C01D92AA30B207CA
:100A3000E1F70E9467160C94E0290C940000FF93E4
:100A4000EF93E0919C01F0919D01309709F0099599
:100A5000EF91FF910895FC018591803011F0EFDF57
:100A6000FBCF0895FF27E0E230E247FF0CC041953D
:100A700097FF09C0EDE26095709580959095611D96
:100A8000711D811D911D27FF02C0219530E350E2A9
:100A9000AA27660F771F881F991FAA1FA41710F097
:100AA000A41B63955A95A9F7AA3008F0A95FA05D29
:100AB000AF93F395611571058105910541F7ED320D
:100AC00011F4EF93F395F21718F43F93F395FBCFDE
:100AD0008F91B5DFFA95E1F70895E991F991859144
:100AE000803021F0853219F0AADFF9CF089520E097
:100AF000E89455915532C1F3503311F468945591EF
:100B00005A3348F4505390F3220F022E220F220F33
:100B1000200D250FF4CF0EF421958991999153362C
:100B200019F3533729F1533559F1BC018827992717
:100B3000E8945C3621F489919991689455915436E2
:100B400039F446EF7EF077FF0DC08FEF9FEF0AC0BC
:100B500055374AE039F0583540E121F0523642E04D
:100B600009F00895FF93EF937DDFEF91FF91B7CFE9
:100B7000FF93EF93FC0181918030B9F360DFFBCFED
:100B8000FF93EF9368DFF1CFDF93CF93CDB7DEB75D
:100B90002596A3DFCF91DF9108950895BF92CF925C
:100BA000DF92EF92FF920F931F93CF93DF93E82E84
:100BB000F62EE901E42FF0E0611106C0E45EFE4F7D
:100BC0008491B82EE82F71C0262F30E0E45EFE4FEE
:100BD000E491FE2FCE2ED12C46E0849FC00111243B
:100BE0000FEF10E0B8010E94A5294BEA4603C001AF
:100BF000479F900D11248E0D911D8E0D911D982FE4
:100C0000990F890FD801A21BB30BAC9DA001AD9D1C
:100C1000500DBC9D500D1124B52EF89ED00111240D
:100C2000AB2FBB277801EA1AFB0AEC9CD001ED9CA4
:100C3000B00DFC9CB00D11247801E81AF108E29E79
:100C4000C001E39E900DF29E900D1124892F9927EB
:100C5000081B190B0C9D90010D9D300D1C9D300D36
:100C60001124832F6230710591F048F461157105EC
:100C7000E1F061307105B9F48E2FEB2F16C06430AE
:100C8000710569F040F06630710579F00CC08E2F67
:100C9000E52FB32E0AC0E52FBF2E8B2F06C0852F60
:100CA000BE2EE32F02C0852FBB2EE9838883BA8234
:100CB000DF91CF911F910F91FF90EF90DF90CF9038
:100CC000BF9008959091370292FF0DC0282F287190
:100CD000283019F4877F846006C0282F24712430BF
:100CE00011F48B7F886093FF0DC0282F2871283165
:100CF00019F4877E846106C0282F2471243111F4F1
:100D00008B7E88612091380220FF0DC0382F38710A
:100D1000383019F4877F816006C0382F3171313047
:100D200011F48E7F886021FF0DC0282F2871283193
:100D300019F4877E816106C0282F2171213111F4B9
:100D40008E7E886194FD877E08951F93CF93DF93F5
:100D5000CDB7DEB767970FB6F894DEBF0FBECDBF35
:100D60004B8B5C8B6D8B7E8B8F8B86E09E01235F24
:100D70003F4FD901E82F1D92EA95E9F795E0FE0172
:100D80007396D90101900D929A95E1F7F901DE0170
:100D9000179601900D928A95E1F7CE0107960E9471
:100DA000E62181113EC086E0FE013796DE011196F4
:100DB00001900D928A95E1F7FF81E8856A857B8530
:100DC0006115710531F0EF3F31F481E0FF3F19F417
:100DD00003C081E001C080E080FD23C02091940227
:100DE00030E0C9010196877099274091C50250E013
:100DF0008417950779F1F983EA837D836C8396E004
:100E0000929FD001939FB00D1124AB56BD4FFE01B0
:100E1000319601900D929A95E1F7809394020E9489
:100E2000702116E08091C502909194028917F9F023
:100E3000189FC00111248B569D4F0E94E6218823E4
:100E4000B1F08091C50290E0019687709927809358
:100E5000C502E8CF0E946727109294021092C50243
:100E6000EEE8F2E086E0DF011D928A95E9F76796E9
:100E70000FB6F894DEBF0FBECDBFDF91CF911F91AB
:100E8000089520912802309129022817390771F01E
:100E90009093290280932802E0913A02F0913B025C
:100EA000309721F00084F185E02D09940895209178
:100EB0002602309127022817390771F090932702F4
:100EC00080932602E0913A02F0913B02309721F0A4
:100ED0000680F781E02D09940895E0913A02F0919F
:100EE0003B02309721F00190F081E02D099480E0E1
:100EF00008950F931F93CF93DF93C62FD42F122FF4
:100F0000FC0182818823C9F060932A020E94A325F4
:100F1000909325028093240280E28C0F883008F0A1
:100F20005EC0C77081E001C0880FCA95EAF7DF9103
:100F3000CF911F910F910C947D2780912A02681305
:100F40003EC080912402909125020E949425883C05
:100F50009105A8F500E20D0FCD17B9F080E28C0FD6
:100F6000883040F4C77081E001C0880FCA95EAF765
:100F70000E947227083048F481E09D2F977001C0CD
:100F8000880F9A95EAF70E947D27812F0E94EE270D
:100F9000193349F4FFEF27EE83E0F1502040804001
:100FA000E1F700C00000812F0E9487270830B8F4C5
:100FB000D77081E001C0880FDA95EAF70AC080E2B5
:100FC0008C0F883060F4C77081E001C0880FCA952B
:100FD000EAF7DF91CF911F910F910C947227DF9167
:100FE000CF911F910F910895882311F0FA0101C04C
:100FF000FB010994109253028091620280FF08C0A5
:1010000087EE92E09F938F930E94C4050F900F90FC
:10101000089580914D0280FF0AC0809A81B38E7F2F
:1010200091B391602FB7F894E4EAF1E00BC0E4EAE1
:10103000F1E0118210821282339631E0E43DF30731
:10104000C1F7EBCF31E0E43DF30789F0319148E09F
:1010500091BB000000C037FF81BB330F000000C010
:1010600000C000C081BB00C04A9591F7EBCF2FBFF5
:101070008FE594E00197F1F700C0000008958F928A
:101080009F92AF92BF92CF92DF92EF92FF920F9317
:101090001F93CF93DF93FC01B280948081E084831F
:1010A000C4EDD1E004EA11E08BE4A82E88248394F7
:1010B000EE24EA94F12C2BE4C22ED12C911003C023
:1010C0001B821A824AC02B81222311F121502B83CB
:1010D0003C81332319F09A2D921B01C0922F8091ED
:1010E0005002899FC0011124B6010E94A5296A837C
:1010F000211104C0332311F01C82AB8222E02B1596
:1011000060F180914E02888380914F02898325C0CF
:101110000E94DE288230914004F582E08B1530F485
:101120000E94DE28B7010E94B92902C080914E02B8
:10113000888322E02B1558F40E94DE2820914F026C
:101140002695622F70E00E94B929820F02C080911B
:101150004F0289831A82AB828C8298014A8169810D
:1011600088810E94CE0525960D5F1F4F82E0C43214
:10117000D80709F0A3CFDF91CF911F910F91FF9076
:10118000EF90DF90CF90BF90AF909F908F900C9496
:101190000908EF92FF920F931F93CF93DF938C0177
:1011A000C4EAD1E0E12CF12CF8018481F8E0EF16DB
:1011B000F1041CF4882339F002C0811104C09E019F
:1011C0004091500202C09E0140E060914F02809128
:1011D0004E020E94CE058FEFE81AF80A239690E19E
:1011E000E916F10409F70E940908F801848190E0EA
:1011F0000196817099278483DF91CF911F910F9180
:10120000FF90EF900895EF92FF920F931F93CF936B
:10121000DF93EC018C819D810196817099279D83DC
:101220008C8384EAE82E81E0F82E10E005E5212F7A
:1012300026958C819D81820F911D8170970140912F
:10124000500260914F02809F802D11240E94CE0594
:101250001F5F83E0E80EF11C103149F7DF91CF9159
:101260001F910F91FF90EF900C9409080F931F931B
:10127000CF93DF93C4EAD1E0FE0111821082128283
:10128000339681E0E43DF807C1F700E010E080917B
:10129000A201082E000C990B0817190794F08091F1
:1012A0001001082E000C990B8017910754F09E0135
:1012B0004091500260914F0280914E020E94CE05F3
:1012C00003C0198218821A820F5F1F4F23960031C4
:1012D0001105E9F60E94090880910F019091A20181
:1012E000980F9093A20120911001280F20931001D4
:1012F000121614F49F301CF0819580930F01DF913A
:10130000CF911F910F910895CF92DF92EF92FF92AC
:101310000F931F93CF93DF93FC01828180FF03C063
:10132000DD24DA9402C0DD24D394C4EAD1E000E0E5
:1013300010E0198218821A8294E0E92EF12CC12C57
:101340008091A1018C0D813114F08F7002C087FD56
:10135000805F082E000C990B0817190791F48091F3
:1013600050028E9DA0018F9D500D112455954795DB
:10137000559547959E0160914F0280914E020E94C3
:10138000CE05CD0CF1E0EF1AF108D1F60F5F1F4F3B
:1013900023960031110569F60E9409088091A10188
:1013A00091E0D91206C0811102C08FE006C08150C1
:1013B00004C090E001968F7099278093A101DF917E
:1013C000CF911F910F91FF90EF90DF90CF900895F4
:1013D000EF92FF921F93CF93DF93EC0184EAE82E04
:1013E00081E0F82E10E08C819701409150026091CD
:1013F0004F02810F0E94CE05115F83E0E80EF11CC1
:10140000103F89F70E9409089A818C8190FF02C0E1
:101410008F5F01C081508C83DF91CF911F91FF902E
:10142000EF90089590914D0290FF0CC0E4EAF1E036
:10143000818360834283339691E0E43DF907C1F7ED
:101440000C94090808950F931F93CF93DF9300D056
:101450001F92CDB7DEB78C018091A30181110AC024
:101460009E012F5F3F4F4FEF6FEF0E94CE058A81A5
:101470008093A301F8018481813051F028F08230FB
:1014800061F44091A3010AC08091A30140E007C02C
:101490006091A30140E080E003C040E080E060E0B4
:1014A0000E94120AF801848190E0019663E070E0E6
:1014B0000E94B92984830F900F900F90DF91CF91F4
:1014C0001F910F910895CF93DF9300D01F92CDB756
:1014D000DEB790914D0290FF0AC09E012F5F3F4FF3
:1014E0000E94CE054B8169818A810E94120A0F9069
:1014F0000F900F90DF91CF910895CF93DF93EC0180
:10150000EDE4F2E0438162818C810E94630A8C8168
:101510008F5F8C83DF91CF910895CF93DF93EC01A0
:10152000EC81F0E0E050FD4F4491EDE4F2E06281A7
:1015300081810E94630A8C818F5F8C83DF91CF91C0
:10154000089580914D02282F269530E02115310510
:1015500019F48170826005C02B32310524F081704E
:10156000846580934D020895CF92DF92EF92FF92AF
:101570006B017C010E94A10AB701A60188E090E0FE
:10158000FF90EF90DF90CF900C9414293F924F92F0
:101590005F926F927F928F929F92AF92BF92CF9203
:1015A000DF92EF92FF920F931F93CF93DF9300D0C0
:1015B0001F92CDB7DEB7182F762E042F422E9091B2
:1015C0004D0290FFB2C0E92FE695AE2FB0E0A45EC9
:1015D000BE4F8C91809352029E7F923061F49E01A7
:1015E0002F5F3F4F812F0E94CE054B8169818A81F9
:1015F0000E94120A60C0823019F4009150025BC050
:10160000863019F410914E0256C08930D9F38931D1
:1016100009F051C0E9518E2F8170582E81E0652C60
:101620006826E695F0E0EE51FD4FC590D49034EA7F
:10163000A32E31E0B32EE12CF12CDD244BEB842ED4
:1016400042E0942EEC9CC001ED9C900DFC9C900D12
:10165000112424E0969587952A95E1F7312E5110B3
:1016600002C0380E01C0381A8091620280FF11C09A
:10167000DF92CF921F926F921F923F92FF92EF9252
:101680009F928F920E94C4050FB6F894DEBF0FBEE2
:10169000CDBF9501402F672D832D0E94CE059FEF72
:1016A000E91AF90A83E0A80EB11C90E1E916F104E9
:1016B00049F60E94090810934E0270924F0200935F
:1016C00050024420E9F060914D0270914E028091E9
:1016D0004F02909150020E94B40A8091620280FFF2
:1016E00024C0809150021F928F9380914F021F92CD
:1016F0008F9380914E021F928F9386E992E00CC0E7
:101700008091620280FF11C01F920F931F927F92FF
:101710001F921F938FE692E09F938F930E94C405C0
:101720000FB6F894DEBF0FBECDBF0F900F900F9095
:10173000DF91CF911F910F91FF90EF90DF90CF90AD
:10174000BF90AF909F908F907F906F905F904F90E1
:101750003F900895EDE4F2E0438128E0421B08F455
:1017600040E021E0628181810C94C60AEDE4F2E060
:10177000438128E0420F08F44FEF21E0628181812C
:101780000C94C60AEDE4F2E0628128E0621B08F4E2
:1017900060E021E0438181810C94C60AEDE4F2E02F
:1017A000628128E0620F08F46FEF21E043818181BC
:1017B0000C94C60AEDE4F2E0818121E0438162816C
:1017C00088500C94C60AEDE4F2E0818121E0438167
:1017D0006281885F0C94C60A80915102882319F0B7
:1017E00081508093510260914D0270914E02809120
:1017F0004F02909150020C94B40A809151028330B0
:1018000018F48F5F8093510260914D0270914E02E7
:1018100080914F02909150020C94B40A90914D0225
:1018200090FF68C09170811102C0926006C08B3237
:1018300010F0946502C0880F982B90934D02662398
:10184000B1F060914D0270914E0280914F029091E3
:1018500050020E94B40A8091620280FF1BC08091F6
:101860004D0286951F928F9383E592E00BC0809185
:10187000620280FF0FC080914D0286951F928F9368
:1018800085E392E09F938F930E94C4050F900F9081
:101890000F900F9060914D02669570E04BE050E024
:1018A00084E091E00E94D329892B19F00E94FA0765
:1018B00015C081E0809353020E94A32590934802B3
:1018C000809347028091620280FF08C08CE192E021
:1018D0009F938F930E94C4050F900F9081E0809397
:1018E0004A0220E04091500260914F0280914E02E6
:1018F0000C94C60A089580914D028695815009F492
:101900008AE261E00C940E0C80914D0286958F5F07
:101910008B3208F081E061E00C940E0C90914D0246
:1019200090FF04C09695981740F003C0811105C040
:1019300090E0961710F40C94840C61E00C940E0C5B
:10194000EDE4F2E083E0808311828FEF8283838372
:10195000148260817181828193810C94B40A7F9298
:101960008F929F92AF92BF92CF92DF92EF92FF92AF
:101970000F931F93CF93DF9307E411E0ADE2B2E042
:1019800027E3A22E22E0B22E812CEE24E394F12C48
:10199000E80189918E01E82FE295EF70F0E021A136
:1019A0008F70A70102C0440F551F8A95E2F7CA0144
:1019B000242B21A322A1742E7094272122A350EA64
:1019C0005A95F1F79CE4C92E91E0D92E60E070E0C1
:1019D00040E050E0E60199906E01292D22952F708C
:1019E00030E0E90128A130E0D92DDF7002C0359543
:1019F0002795DA95E2F720FD08C09701062E02C070
:101A0000220F331F0A94E2F702C020E030E0422B9D
:101A1000532B6F5F7F4F6F307105E1F691A1D72D8A
:101A2000D923D1A392A1892B82A38D919C91119747
:101A30004817590729F011965C934E9381E001C035
:101A400080E0882A1296AA16BB0609F0A1CF88204A
:101A500049F081E08093A0010E94A32590939F010B
:101A600080939E018091A001882391F180919E0135
:101A700090919F010E949425069750F180912D022C
:101A800090912E0290933E0280933D0280912F020E
:101A9000909130029093400280933F0280913102F6
:101AA00090913202909342028093410280913302DE
:101AB00090913402909344028093430280913502C6
:101AC0009091360290934602809345021092A001B5
:101AD000882DDF91CF911F910F91FF90EF90DF90B4
:101AE000CF90BF90AF909F908F907F900895CF93AD
:101AF000DF932BE4829FC0011124FC013FE0739F20
:101B0000E00DF11D1124E60FF11DEE0FFF1FE7534D
:101B1000FB4FC591D491CE01C238D10569F1B0F423
:101B2000C133D10509F475C048F4C932D10509F4AF
:101B300069C0CA32D10509F473C085C0C533D10567
:101B400009F459C0C933D105B9F07DC0C33ED105F0
:101B500071F138F4C03ED105B1F0C23ED10511F1AA
:101B600072C0C63ED105B9F1C73ED105C9F1C43E28
:101B7000D10509F068C024C02091370220FD5DC066
:101B800021FD5BC060C02091370220FD50C0209134
:101B9000380220FF67C18091370284FD61C183EE66
:101BA00090E060C12091370222FF5CC1F4CF8091A8
:101BB000370282FD3FC08091380280FD3EC0EBCFEE
:101BC0002091380221FF4EC18091370284FD48C127
:101BD00087EE90E047C12091370223FF43C1F4CF45
:101BE0008091370283FD2CC08091380281FFECCFB9
:101BF00084EE90E037C12091370225FF33C189E29E
:101C000090E030C12091370225FF2CC185E390E0A0
:101C100029C12091370226FF25C18AE290E022C126
:101C20002091370226FF1EC181E390E01BC189E3AA
:101C300090E018C182EE90E015C180EE90E012C1F4
:101C400086EE90E00FC1C11530E5D30708F067C0FC
:101C5000C11540E4D40720F0CE019F70906A02C104
:101C6000C83ED105B8F5C03ED10508F0FBC0C83A62
:101C7000D105B8F4C53AD10550F08C2F855AE82F1C
:101C8000F0E0E659FE4F808190E09064EBC0C130F7
:101C9000D10509F4E7C008F4E3C0249708F4E0C0D4
:101CA000E1C0CF3BD10560F48C2F885AE82FF0E0DB
:101CB000EE0FFF1FE359FE4F808191819464D2C0E3
:101CC000C03CD10508F4CCC0FE01EE0FFF1FE45666
:101CD000F0400EC0C11520E2D20768F0C11540E304
:101CE000D407A8F4FE01FF70EE0FFF1FE45EFE4F65
:101CF00085919491B7C0C11531E0D30708F0B2C007
:101D0000C03FD10508F4ACC0CE019065ABC0CE0198
:101D10009927D3FF02C0986CA5C0906CA3C0C115D1
:101D200085E5D80708F05BC0C11524E5D20728F087
:101D30009C2F8827846F906A95C0C11532E5D30720
:101D400038F5C11541E5D407F0F4CE0174E096955D
:101D500087957A95E1F7282F23703C2F337081E027
:101D600090E002C0880F991F3A95E2F79C68922B89
:101D7000EC2FEF70E695E69540E2E49FF001112428
:101D80008E2B9F2B6FC09C2F8827816F906A6AC013
:101D9000AE01437055272C2F26952695C115D345A6
:101DA00078F481E090E002C0880F991F4A95E2F72D
:101DB00040E2249F90011124822B932B9C6852C0F7
:101DC00081E090E002C0880F991F4A95E2F740E257
:101DD000249F90011124822B932B9A6843C0C11534
:101DE00029E5D207B0F4C11538E5D30728F09C2FB8
:101DF0008827806F906A36C0C11546E5D40780F504
:101E00008C2F0E9462068F7190E0982F8827906235
:101E100029C0C1158AE5D80790F48C2F8F700E94D5
:101E20006206FE0194E0F695E7959A95E1F7EF706A
:101E3000F0E0FE2FEE27F0699F01282B0FC0CE01A6
:101E400090568115904260F48D2F8F710E9462062A
:101E5000FE01FF27F0628F719F01382BC90102C07C
:101E600080E090E0DF91CF9108958F929F92AF92A2
:101E7000BF92CF92DF92EF92FF920F931F93CF9377
:101E8000DF93CDB7DEB72A970FB6F894DEBF0FBE4B
:101E9000CDBFFC010081D18083819481892B39F0F1
:101EA0001FEFD11206C091E00F3F19F403C091E07B
:101EB00001C090E090FDA8C57F0185E0DE01169687
:101EC00001900D928A95E1F7F70122818E819F8121
:101ED000222349F00E945920182F682F8E819F815C
:101EE0000E94D22003C00E94A620182F2BE4129F2C
:101EF000F00111243FE0D39EE00DF11D1124E00F0D
:101F0000F11DEE0FFF1FE753FB4F05911491033FA7
:101F10008CE5180729F180F4083DECE51E07C9F0AF
:101F2000093DFCE51F0741F1073D2CE5120739F596
:101F300026E241EE61EE10C0053F3CE51307C1F01B
:101F400098F0063F9CE51907D1F427E245EE66EECE
:101F500003C027E245EE65EEC7010E94790773C210
:101F600026E241EE60EEF8CF27E245EE64EEF4CFD4
:101F700026E241EE62EEF0CF28E241E0ECCFF7013D
:101F80009281992309F43FC110922A020230FCE5A4
:101F90001F0708F422C106312CE5120738F098011A
:101FA0002A5F3C452930310508F017C10E94972669
:101FB000909338028093370200313CE5130709F40F
:101FC000C3C008F041C008309CE5190709F49AC065
:101FD000F0F40430FCE51F0709F487C068F4023010
:101FE0003CE5130709F477C003301C4509F0E5C050
:101FF00080913702826076C006309CE5190709F4AB
:102000006EC008F07BC08091370288606BC00C30D6
:10201000FCE51F0709F485C068F40A303CE51307A6
:1020200009F474C008F079C00E94672780913702D4
:10203000806858C00E309CE5190709F476C008F096
:102040007FC0809137028BC00B3FFCE51F0709F46E
:102050004FC018F503313CE5130709F47DC078F44F
:1020600001319CE5190709F473C002311C4509F0E0
:10207000A4C00E946727809137028F7733C0053153
:10208000FCE51F0709F472C008F486C00A3F1C452E
:1020900009F093C0809138023EC00F3F8CE51807CD
:1020A00009F45FC058F40D3FECE51E0709F444C085
:1020B00008F43FC08091380282602DC001302DE5C8
:1020C000120709F475C008F45DC002301D4509F01F
:1020D00074C060E06EC080913702816003C080915F
:1020E000370280618093370268C08091370211C047
:1020F000809138028260809338025FC080913702FD
:102100008062F0CF809137028064ECCF80913702FB
:1021100088608460E7CF8160EECF809137028E7F48
:10212000E1CF809137028D7FDDCF80913702877FAD
:10213000D9CF8091380218C0809138028D7FDBCFD3
:10214000809137028F7ECECF809137028F7DCACFAC
:10215000809137028F7BC6CF80913702877F8B7F3C
:10216000C1CF809138028D7F8E7FC5CF809137029D
:1021700082FB222720F991E0922790FB82F990FBC5
:1021800083F9B0CF80913802982F909591708E7F0F
:10219000892B90FB81F9AFCF0E946727809137028E
:1021A00087FB222720F991E0922790FB87F99ACFAD
:1021B00061E08EE090E00E94022960913702109168
:1021C000380284E090E00E940229612F81E290E0D1
:1021D0000E9402290E94672736C18091FF020631C2
:1021E0002CE5120709F58A7A91E009F490E09093C2
:1021F0002B02882311F065E301C069E286E892E0D2
:102200000E947D260EC006311C4509F03BC180911D
:102210002B02882309F4F6C365E386E892E00E9466
:1022200070260E94EF1F0FC18272F801E25CFC452C
:10223000E431F10508F0B6C0EA5AFF4F0C94CD29FD
:102240008091620280FF10C080914D028095817064
:102250001F928F938FE694E09F938F930E94C40503
:102260000F900F900F900F9080914D0280FF2EC025
:102270008E7F80934D0260914D0270914E0280914D
:102280004F02909150020E94B40A8091620280FF36
:102290000FC080914D0281701F928F9380E094E077
:1022A0009F938F930E94C4050F900F900F900F90F3
:1022B0000E94FA079FEFE0E7F2E09150E040F04023
:1022C000E1F700C000000E940908BDC08160809352
:1022D0004D028091620280FF0DC01F9281E08F93BA
:1022E00088E394E09F938F930E94C4050F900F9012
:1022F0000F900F9080914D0261E0869550C04BE7A2
:102300005CE064E87CE02CC044E85CE06BE77CE0E7
:1023100027C04AED5BE063EE7BE022C043EE5BE06A
:102320006AED7BE01DC042EC5BE06EEC7BE018C028
:102330004EEC5BE062EC7BE013C04AEA5BE066EBEC
:102340007BE00EC046EB5BE06AEA7BE009C04CEE46
:102350005BE06DEF7BE004C04DEF5BE06CEE7BE09B
:102360000E94F40770C061E081E019C065E082E07E
:1023700011C068E086E00EC06EE089E00BC064E149
:102380008FE008C067E185E105C061E088E107C032
:1023900062E289E10E948E0C56C061E083E20E94F5
:1023A0000E0C51C001302CE51207C1F10E3D3CE589
:1023B000130709F446C001151C4509F063C00E94CB
:1023C00067279FEFE4E3FCE09150E040F040E1F745
:1023D00000C0000081E08093E00080E28093D8009C
:1023E0001092C9008FE19EE40197F1F700C0000050
:1023F00087E090EBDC0180930A0390930B03A0939A
:102400000C03B0930D039CE088E10FB6F894A895F7
:10241000809360000FBE90936000FFCF80916202B6
:10242000982F9095917090FB80F980936202992388
:1024300019F088EB94E002C086EA94E00E942B0534
:1024400002C00E94A8268091FC02877009F4DCC2B9
:10245000F7018281882309F4D7C282E02A960FB659
:10246000F894DEBF0FBECDBFDF91CF911F910F91CA
:10247000FF90EF90DF90CF90BF90AF909F908F90A4
:102480000C942C21F70100811181992349F0C80196
:102490000E945920D82E682FC8010E94D22004C063
:1024A000C8010E94A620D82EB8018D2D0E94770D5C
:1024B0008C01982EF701A580A2942FE0A222D28051
:1024C000D1101092FE028091FC02877099F0DD20FD
:1024D00089F0812F807F803421F080E2800F883066
:1024E00048F082E00E942C218091FC028770CC246D
:1024F000C3948111C12CB12EB2949FE0B9228B2DCF
:1025000090E08C30910508F040C2FC01E659FF4F85
:102510000C94CD29812F807F1F70882311F0129594
:10252000107FDD20B9F0112309F41AC280E2800F78
:10253000883010F0911006C08091FF02182B109384
:10254000FF0205C08091FE02182B1093FE020E942C
:10255000EF1F06C2802F0E948727112309F415C29E
:10256000005E1095083010F0911006C08091FF02B7
:1025700018231093FF0205C08091FE0218231093C8
:10258000FE020E94EF1F01C2812F807F1F708032E8
:1025900011F01295107F992021F0F1E09F16E1F0E3
:1025A0002AC0DD2081F080910003AA2051F001E0D3
:1025B000A01207C0182B181709F4E7C110930003E5
:1025C000E4C1812B10C0AA2021F021E0A21609F459
:1025D000DCC10E941D2727C0DD2041F035E03A15FF
:1025E00008F4D3C1812F0E947D27CFC184E08A15D2
:1025F00008F4CBC118C0DD2049F0AA2099F3F701F7
:10260000858180FFADC18F708583ECCFAA2059F002
:10261000093309F0B7C1FFEF17EE23E0F150104086
:102620002040E1F7ADC1812F0E947227AEC1812FFA
:1026300086958695837019F0813059F0A6C1DD200A
:1026400019F0C801937002C080E090E00E94570723
:10265000A2C1DD2019F0C801937002C080E090E0B3
:102660000E94410798C1802FDD2019F00E940625A5
:1026700002C00E943F240E94AF258DC1812F83702C
:1026800009F069C0D11085C1902F929596959770E9
:10269000990F990F802F8F70882E912CA12CB12C1F
:1026A000092E04C0880C991CAA1CBB1C0A94D2F7E2
:1026B00004FF12C04FE050E060E070E004C0440F3F
:1026C000551F661F771F9A95D2F7DB01CA018095C7
:1026D0009095A095B09503C080E090E0DC01169540
:1026E0001695412F4370423019F1C8F4009101034F
:1026F000109102032091030330910403413059F0FB
:1027000088299929AA29BB29BC01CD0160237123FD
:10271000822393230AC0802A912AA22AB32ABC01C9
:10272000CD01682979298A299B290E94662131C116
:1027300088299929AA29BB29009101031091020334
:102740002091030330910403BC01CD016027712760
:1027500082279327EACFDD2019F0812F817001C0F5
:102760008695882309F415C1902F929596959770B8
:10277000990F990F802F8F70882E912CA12CB12C3E
:10278000092E04C0880C991CAA1CBB1C0A94D2F701
:1027900004FF12C04FE050E060E070E004C0440F5E
:1027A000551F661F771F9A95D2F7DB01CA018095E6
:1027B0009095A095B09503C080E090E0DC0116955F
:1027C0001695412F43704230D9F068F50091F80218
:1027D0001091F9022091FA023091FB02413059F038
:1027E00088299929AA29BB29BC01CD01602371231D
:1027F000822393231EC0802A912AA22AB32A13C0BF
:1028000088299929AA29BB290091F8021091F90277
:102810002091FA023091FB02BC01CD0160277127A3
:102820008227932706C0BC01CD01682979298A290E
:102830009B290E94FD20ADC01F70DD2039F0812F43
:102840000E944521802F0E947D27A3C0802F0E94D7
:102850007227812F0E9407219CC0802F32EF931690
:1028600009F440C0391538F090EF991661F0E1EFA6
:102870009E1699F170C0F3EF9F16D9F124EF9216CE
:1028800009F44EC068C0DD2019F134E03A1508F4AF
:102890007CC01F7181E090E0A0E0B0E0AC01BD0120
:1028A00004C0440F551F661F771F1A95D2F78091F9
:1028B000F8029091F902A091FA02B091FB028A010C
:1028C0009B01082719272A273B27C901B80125C0E2
:1028D00025E02A1508F459C0DCCFDD2029F0812F2E
:1028E0008F712CC0DD20D9F3812F8F710E940721B9
:1028F0004CC0DD2079F01F7181E090E0A0E0B0E0F5
:10290000BC01CD0104C0660F771F881F991F1A955F
:10291000D2F703C060E070E0CB010E94FD2035C01B
:10292000DD2079F01F71812F0E94452138E0139F2F
:10293000C001112483608093FC02812F0E944521F5
:1029400024C081E00E942C2181E08A15F0F482E00D
:102950000E942C211AC0DD2039F0AA2009F4BFCF33
:10296000802F0E94EE2711C0AA2009F4BDCF893321
:1029700049F49FEFE7EEF3E09150E040F040E1F7DB
:1029800000C00000802F0E94872788EF8B0D8430C5
:1029900010F40E946D07CC20A9F08091FC0280FD0C
:1029A00011C0F70112828595859585950E94452174
:1029B000C7010E94350F8091FC028595859585950C
:1029C0000E94072185E0F701DE01119601900D922A
:1029D0008A95E1F789819A810E94A6209A810BE469
:1029E000809FF00111241FE0919FE00DF11D112443
:1029F0008981E80FF11DEE0FFF1FE753FB4F859113
:102A0000949102C069E209CC2A960FB6F894DEBF11
:102A10000FBECDBFDF91CF911F910F91FF90EF902F
:102A2000DF90CF90BF90AF909F908F9008959FB709
:102A3000F89410926D029FBF90917C02943009F03F
:102A400057C09091E9009F703091EC00232F2170C6
:102A500030FD20E8922B23E02093E9002091EB0049
:102A600020FF43C02091EE0027FF3FC020912C02A1
:102A7000222321F02091E80025FF37C010922C027C
:102A800026E03091E80035FD15C030917C023430ED
:102A900061F53091EB0035FD28C0215021F481E033
:102AA00080932C0222C0EFE9FFE03197F1F700C0DC
:102AB0000000E7CF8093F1008091E80085FD0AC017
:102AC0008091E80080FFFCCF8091E8008E778093B2
:102AD000E80006C08FB7F89421E020936D028FBF05
:102AE0009F709093E90080E008959F709093E900B3
:102AF0008FEF08952091E4003091E50095E6409134
:102B0000EC00842F817040FF23C08091E80080FD9D
:102B10001DC080917C02882399F0853099F08091C6
:102B2000EB0085FD11C04091E4005091E5002417B1
:102B3000350729F3915011F09A01E1CF84E008950F
:102B400082E0089583E0089581E0089580E008958B
:102B50004091E80042FFDDCF089580917E0287FF1B
:102B600011C08091E80082FD05C080917C02811136
:102B7000F8CF11C08091E8008B770BC080917C0268
:102B8000882349F08091E80080FFF8CF8091E80029
:102B90008E778093E8000895982F973068F590938A
:102BA000E900981739F07091EC002091ED005091F8
:102BB000F00003C0242F762F50E021FD02C09F5F5C
:102BC000ECCF3091EB003E7F3093EB003091ED0085
:102BD0003D7F3093ED003091EB0031603093EB009E
:102BE0007093EC002093ED005093F0002091EE00E4
:102BF00027FDE5CF80E008958F708093E90081E0A4
:102C0000089520918402309185022617370748F0F5
:102C10006115710539F42091E8002E772093E800C2
:102C200001C0B901FC0120E06115710579F18091C5
:102C30007C028823F1F18530F1F18091E80083FD79
:102C40003CC08091E80082FD2EC08091E80080FFAA
:102C5000EBCF2091F3008091F20090E0922B611570
:102C6000710551F08830910538F421912093F100DD
:102C7000615071090196F3CF21E0089709F020E037
:102C80008091E8008E778093E800CECF2111CFCFDE
:102C90000AC080917C02882361F0853061F08091C8
:102CA000E80083FD0AC08091E80082FFF2CF80E057
:102CB000089582E0089583E0089581E00895809169
:102CC0007C02843011F081E0089582E00895CF9372
:102CD000DF93CDB7DEB761970FB6F894DEBF0FBEB6
:102CE000CDBF84B7877F84BF0FB6F894A895809135
:102CF0006000886180936000109260000FBE90E0D9
:102D000080E80FB6F89480936100909361000FBE45
:102D100085B7806885BF85B7806885BF0E94421EE1
:102D20000E94611E8091E20084608093E20087E14E
:102D300095E190939D0180939C01789480917C0211
:102D40008823A1F01091E9001F709091EC00892F69
:102D5000817090FD80E8182B1092E9008091E800C6
:102D600083FD0E94271B1F701093E90082E084BD41
:102D700093E095BD9AEF97BD80936E00A7E4B1E014
:102D800041E050E08D91E82FE295EF70F0E021A155
:102D90008F708A0102C0000F111F8A95E2F7C801E7
:102DA000902F9095922391A392A1892B82A311E059
:102DB000AC34B10739F7ACE4B1E04BE551E061E088
:102DC00070E08D91E82FE295EF70F0E021A18F7017
:102DD0008B0102C0000F111F8A95E2F7C801902FE6
:102DE0009095922391A392A1892B82A34A175B0706
:102DF00041F7EDE2F2E0ADE3B2E0119211921D92E3
:102E00001D9212E0E733F107C1F780E090E00E94E5
:102E1000FC288C3E9E4F11F00E94A82680E090E096
:102E20000E94FC288C3E9E4F11F00E94A82682E052
:102E300090E00E94EE28809362020E949726909371
:102E400038028093370283E090E00E94EE28682FDA
:102E500070E080E090E00E9466218091390281114B
:102E6000E0C08091620280FF08C087E397E09F93F3
:102E70008F930E94C4050F900F908091620280FF93
:102E800008C081E297E09F938F930E94C4050F9042
:102E90000F9080E090E00E94FC288C3E9E4F81F0D5
:102EA0008091620280FF08C089EF96E09F938F9324
:102EB0000E94C4050F900F900E94A8260E94A00CAB
:102EC00088E090E00E94F62860934D0270934E02D5
:102ED00080934F02909350026E7FD1F480916202F2
:102EE00080FF08C080EB96E09F938F930E94C405FB
:102EF0000F900F900E94A00C88E090E00E94F628AE
:102F000060934D0270934E0280934F029093500253
:102F10000E94A10A8091620280FF08C087E996E0C2
:102F20009F938F930E94C4050F900F90809162022F
:102F300080FF0FC080914D0281701F928F938AE7AE
:102F400096E09F938F930E94C4050F900F900F906F
:102F50000F908091620280FF0FC080914D02869594
:102F60001F928F938FE596E09F938F930E94C405E5
:102F70000F900F900F900F908091620280FF0EC013
:102F800080914E021F928F9385E496E09F938F93DA
:102F90000E94C4050F900F900F900F9080916202D5
:102FA00080FF0EC080914F021F928F938BE296E0BC
:102FB0009F938F930E94C4050F900F900F900F90D6
:102FC0008091620280FF0EC0809150021F928F9309
:102FD00081E196E09F938F930E94C4050F900F901C
:102FE0000F900F908091620280FF0EC0809151027D
:102FF0001F928F9385EF95E09F938F930E94C40556
:103000000F900F900F900F901092530280914D02ED
:1030100080FF04C060E086950E940E0C81E08093E2
:10302000390281E191E090933B0280933A0288EA71
:1030300097E00E942B0580917C02853009F03FC00B
:1030400084EA97E00E942B0580917C02843021F174
:1030500010923C0220E488E190E00FB6F894A89525
:10306000809360000FBE2093600083B7817F8460EF
:1030700083BF83B7816083BF7894889583B78E7F41
:1030800083BF0FB6F894A895809160008861809303
:103090006000109260000FBE80917B02882309F4CB
:1030A000CACF0E94AF0CEDE3F2E081919191892BA0
:1030B00009F081C252E0E734F507B9F7BCCF0E94AE
:1030C000AF0C43E6642E42E0742E5DE3452E52E0E1
:1030D000552E00E010E0098BF201A190B1902F0174
:1030E000F301C190D1903F01CA24DB24C114D10463
:1030F000B1F40F5F1F4F0530110569F78FEF8C8713
:103100008D871E860E94A3258160782F988B8F87DC
:103110004C855D856E8588890E94A50677C0809163
:10312000620281FD05C080E0EE24E394F12C48C0EA
:103130008EE597E00E942B052DE3822E22E0922E51
:10314000E12CF12CFF92EF9229E537E03F932F938A
:103150000E94C40586E597E00E942B05F40180815A
:103160002180F2E08F0E911C0E940B27382E822DB9
:103170000E940B27232D30E0322F2227A901482B54
:10318000CA019F938F9360E577E07F936F930E94CE
:10319000C4058EE497E00E942B059FEFE91AF90A17
:1031A0000FB6F894DEBF0FBECDBFF5E0EF16F10409
:1031B00049F6B9CF8F5FEE0CFF1C8F3009F499CF21
:1031C00096012E213F21232BA9F38F83298928875C
:1031D000AE20BF2081E0AB2809F480E089870E94FF
:1031E000A3258160782F9B878A874F8158856985C1
:1031F0008B850E94A506000F111FF801ED59FD4FA8
:1032000080819181E826F926F182E0828091530243
:10321000882309F4ACC080915202E0914D02E695FA
:10322000E81BE0934902823059F4F0E0EA57F84F86
:10323000E4910E2F10E0FDE8EF2EFAE0FF2E6BC0B8
:10324000863059F4F0E0ED57F84FE4910E2F10E07E
:10325000EDE7EE2EEAE0FE2E5EC0893061F4E695E1
:10326000F0E0E058F84FE4910E2F10E078EEE72EF2
:1032700079E0F72E50C08F3061F4E695F0E0E35826
:10328000F84FE4910E2F10E064E8E62E69E0F62E88
:1032900042C0853159F4F0E0E658F84FE4910E2F22
:1032A00010E056E3E52E59E0F52E35C08831F9F0EF
:1032B000833249F4E8E7F7E00591149143E2E42E04
:1032C0004AE0F42E28C08432C9F08532F1F48E2F02
:1032D00063E00E949929E92FF0E0EB58F84FE49160
:1032E0000E2F10E03FE3E32E38E0F32E14C008EE7B
:1032F00013E023E0E22E29E0F22E0DC004EF11E0EE
:1033000099ECE92E98E0F92E06C000ED17E08DEC5F
:10331000E82E85E0F82E80914A02882389F01092E9
:103320004A020E94A325980120953095820F931F91
:10333000909348028093470210924C0210924B02E5
:1033400080914702909148020E949425801791072E
:1033500070F0E0914702F09148020E0F1F1F10938A
:1033600048020093470287E492E0F701099586E05E
:10337000EBE5F2E0DE01119601900D928A95E1F7FE
:1033800080915D02811105C080915E02882309F45D
:103390006EC08091590290915A020E9494259C011E
:1033A00090915802992309F41CC12333310508F484
:1033B0005EC09F3F19F09F5F9093580210925F028A
:1033C0001092600280915D02181624F40E94E62497
:1033D00080935D0280915D0287FF05C00E94E62414
:1033E000819580935D0280915E02181624F40E94FC
:1033F000E62480935E0280915E0287FF05C00E94F2
:10340000E624819580935E0230915D023323E1F0E2
:1034100020915E022223C1F005EB3003C00111248C
:10342000992319F090935D0203C081E080935D02BF
:1034300015EB2103C0011124992319F090935E022A
:1034400003C081E080935E020E94AF258091560206
:103450009091570290935A028093590286E0FE01A0
:103460003196ABE5B2E001900D928A95E1F780913B
:103470005F02811105C080916002882309F46EC04B
:1034800080915402909155020E9494259C01909144
:103490005802992309F4AAC02536310508F45EC004
:1034A0009F3F19F09F5F9093580210925D02109217
:1034B0005E0280915F02181624F40E94C424809357
:1034C0005F0280915F0287FF05C00E94C42481953E
:1034D00080935F0280916002181624F40E94C42435
:1034E000809360028091600287FF05C00E94C4241F
:1034F00081958093600230915F023323E1F0209147
:1035000060022223C1F045EB3403C001112499234A
:1035100019F090935F0203C081E080935F0255EB46
:103520002503C0011124992319F09093600203C070
:1035300081E0809360020E94AF25809156029091B5
:103540005702909355028093540286E0FE01319613
:10355000ABE5B2E001900D928A95E1F70E946D070C
:1035600090916102891709F466CD0E946D07182FAA
:10357000809361028091620282FF5DCD80FF04C072
:1035800081E997E00E942B058091620280FF0CC0C8
:103590001F921F936CE877E07F936F930E94C4059E
:1035A0000F900F900F900F908091620280FF43CD9B
:1035B0008AE897E03ECD80E189BD82E189BD09B40A
:1035C00000FEFDCF8091D8008F7D8093D800809140
:1035D000E00082608093E0008091E00081FDFCCFFC
:1035E0002ACD2D32314008F0E6CE41CF2D32314088
:1035F00008F058CFB3CFEF92FF920F931F93CF9362
:10360000DF937C018B010E947A15811119C0E701BB
:1036100001151105A1F08091E80085FD0AC0809197
:10362000E8008E778093E8000E947A15882381F362
:1036300007C089918093F10001501109E9CF80E022
:10364000DF91CF911F910F91FF90EF9008951F93FD
:10365000CF93DF93CDB7DEB7AA970FB6F894DEBF4E
:103660000FBECDBFEEE7F2E086E892E02091F100D8
:1036700021938E179F07D1F780917F02833009F441
:1036800060C030F4813071F0823009F49AC0B1C06A
:103690008A3009F486C08B3009F46BC0893009F098
:1036A000A8C020C080917E02813A09F0A2C080911A
:1036B000E800877F8093E8008091820290918302E6
:1036C000892B21F468E082E792E003C060E080E0AB
:1036D00090E070E00E9401168091E8008B77809363
:1036E000E80087C080917E02813209F082C080911B
:1036F000820290918302029708F07BC08091E800DB
:10370000877F8093E8008091E80082FD05C080916A
:103710007C028111F8CF6DC02091F3008091F200FE
:1037200090E0922B029729F48091F1008B7F8130F9
:1037300021F48091F100809371028091E8008B77F1
:1037400054C080917E02813A09F053C08091820278
:1037500090918302892B09F04CC08091E800877F0B
:103760008093E8008091E80080FFFCCF80911B01EE
:1037700037C080917E028132E1F580918202909182
:103780008302892BB1F58091E800877F8093E80060
:103790000E94AD158091800280931B010E946727D3
:1037A00028C080917E02813221F58091E800877FD8
:1037B0008093E8000E94AD15809181028093700291
:1037C00018C080917E02813AA1F48091E800877F41
:1037D0008093E8008091E80080FFFCCF8091700228
:1037E0008093F1008091E8008E778093E8000E943A
:1037F000AD158091E80083FFE3C180917E02909136
:103800007F02492F50E04A30510508F0D9C1FA0132
:10381000EA58FF4F0C94CD29803821F0823809F006
:10382000CFC108C080917A0290917B02992389F0E0
:1038300082600FC0809182028F70873008F0C0C113
:103840008093E9008091EB0085FB882780F9109236
:10385000E9009091E800977F9093E8008093F10051
:103860001092F1007BC1282F2D7F09F0A9C1882378
:1038700019F0823061F0A4C180918002813009F09A
:103880009FC1933009F080E080937B022EC080912D
:10389000800281112AC0809182028F702FEF280F41
:1038A000263008F08DC18093E9002091EB0020FFC5
:1038B0001CC0933021F48091EB00806214C0909181
:1038C000EB0090619093EB0021E030E0A90102C091
:1038D000440F551F8A95E2F74093EA001092EA00E0
:1038E0008091EB0088608093EB001092E90080915A
:1038F000E800877F8093E8000E94AD1561C18111C7
:103900005FC1109180021F778091E3008078812B46
:103910008093E3008091E800877F8093E8000E9415
:10392000AD158091E80080FFFCCF8091E3008068B6
:103930008093E300111102C082E001C083E0809314
:103940007C023EC18058823008F03AC1209180024A
:10395000309181022C3D53E0350779F583E08A836D
:103960008AE289834FB7F894DE01139620E03EE0A7
:1039700051E2E32FF0E050935700E49120FF03C0A1
:10398000E295EF703F5FEF708E2F90E0EA3010F01D
:10399000C79601C0C0968D939D932F5F243149F740
:1039A0004FBF8091E800877F8093E8006AE270E073
:1039B000CE0101960E940116C0C0809182029091B2
:1039C0008302432F552743305105B1F068F441304D
:1039D000510509F404C14230510509F0F1C08BE5ED
:1039E00090E0E0EBF8E057C04132510589F14232F6
:1039F000510509F43CC0E4C0C90199278130910503
:103A0000B9F070F082309105D9F0039709F0D8C071
:103A1000EDE1F9E0E4918E2F90E0EDE1F9E038C0BE
:103A2000E3E4F9E0E4918E2F90E0E3E4F9E030C0C4
:103A3000E1E3F9E0E4918E2F90E0E1E3F9E028C0C2
:103A4000E3E2F9E0E4918E2F90E0E3E2F9E020C0B8
:103A50008330910508F0B4C0880F991FFC01EC5920
:103A6000FE4F0190F081E02D89E090E014C083309A
:103A7000910508F0A5C0FC01EE0FFF1FE25AFE4FB2
:103A80000190F081E02DDC01A55ABE4F8C9190E0B1
:103A9000009709F495C02091E800277F2093E80063
:103AA00020918402309185022817390708F4C90152
:103AB00040E0009789F120917C02222309F43DC067
:103AC0002530D9F12091E80023FD37C02091E8008E
:103AD00022FD2FC02091E80020FFEBCF4091F300A2
:103AE0002091F20030E0342B009759F02830310556
:103AF00040F444914093F100319601972F5F3F4F7E
:103B0000F3CF41E02830310509F040E02091E80092
:103B10002E772093E800CDCF4111CDCF0AC0809100
:103B20007C02882351F0853041F08091E80083FDCC
:103B300004C08091E80082FFF2CF8091E8008B778B
:103B40008093E8003DC08038D9F58091E800877FF8
:103B50008093E80080917D028093F1008091E800DD
:103B60008E77C8CE81112CC0809180029091810205
:103B7000992702972CF58091E800877F8093E800D1
:103B80001091800210937D020E94AD15111106C0A4
:103B90008091E30087FD02C081E001C084E0809352
:103BA0007C0242E061EC81E00E94CC1542E261ECD3
:103BB00082E00E94CC1542E261EC83E00E94CC15C9
:103BC0008091E80083FF10C08091E800877F809398
:103BD000E8008091EB0080628093EB0005C082E1F9
:103BE00090E0EBE0F9E057CFAA960FB6F894DEBF6D
:103BF0000FBECDBFDF91CF911F9108951F920F92FD
:103C00000FB60F9211242F933F934F935F936F93AF
:103C10007F938F939F93AF93BF93CF93DF93EF9354
:103C2000FF93C091E900CF708091EC00D82FD17044
:103C300080FDD0E81092E9008091F000877F8093AA
:103C4000F00078940E94271B1092E9008091F00008
:103C500088608093F000CD2BCF70C093E900FF9176
:103C6000EF91DF91CF91BF91AF919F918F917F9114
:103C70006F915F914F913F912F910F900FBE0F90D9
:103C80001F901895E8EDF0E080818E7F8083109280
:103C9000E2001092DA001092E100A0EEB0E08C9108
:103CA00081608C9380818F77808319BCA7EDB0E011
:103CB0008C918E7F8C9380818F7E808310926F0297
:103CC0000895CF92DF92EF92FF920F931F93CF93BD
:103CD000DF93C8EDD0E088818F7E8883E7EDF0E048
:103CE00080818160808384E082BF81E080936F0265
:103CF00088818E7F888302EE10E0F8011082109296
:103D0000DA0081EEC82ED12CF601108288818F77DF
:103D1000888388818068888388818F7D888319BCA7
:103D200010927C0210927D0210927B0210927A0215
:103D300090EEE92EF12CF70180818B7F80838881C2
:103D40008160888342E060E080E00E94CC15F6014B
:103D500080818E7F8083F801808181608083808173
:103D600088608083F70180818E7F80838881806175
:103D70008883DF91CF911F910F91FF90EF90DF909B
:103D8000CF9008951F920F920FB60F9211242F9388
:103D90003F934F935F936F937F938F939F93AF93D3
:103DA000BF93EF93FF938091E10082FF49C0809120
:103DB000E20082FF45C08091E1008B7F8093E100AB
:103DC00020916E022F5F822F62E30E94992999232E
:103DD00019F020936E0234C010926E0280916D0231
:103DE000882371F180917C02843041F58091E90053
:103DF0008F702091EC00922F917020FD90E8892B1C
:103E000093E09093E9009091EB0090FF14C09091A3
:103E1000EE0097FF10C09091E80095FF03C010924C
:103E2000F100F9CF9091E80090FF05C09091E80073
:103E30009E779093E8008F708093E90010926D0256
:103E40008091DA0080FF32C08091D80080FF2EC0C0
:103E50008091DA008E7F8093DA008091D90080FF14
:103E60001CC080E189BD82E189BD09B400FEFDCF9F
:103E700081E080937C028CE998E00E942B05809180
